:0200000480007A
:100000006F008004732F2034930F80006308FF0378
:10001000930F90006304FF03930FB0006300FF038E
:10002000130F000063040F0067000F00732F2034CC
:1000300063540F006F00400093E19153171F0000BD
:1000400023223FFC6FF09FFF93000000130100008C
:10005000930100001302000093020000130300004C
:100060009303000013040000930400001305000034
:10007000930500001306000093060000130700001C
:100080009307000013080000930800001309000004
:1000900093090000130A0000930A0000130B0000EC
:1000A000930B0000130C0000930C0000130D0000D4
:1000B000930D0000130E0000930E0000130F0000BC
:1000C000930F0000732540F16310050097020000B4
:1000D000938202017390523073500018970200000F
:1000E00093824202739052309B021000939252030B
:1000F0009382F2FF7390023B9302F0017390023AF5
:100100007350403097020000938242017390523046
:10011000735020307350303093010000970200007C
:10012000938282EE73905230130510001315F5017F
:10013000635C05000F00F00F930110009308D005D9
:10014000130500007300000093020000638A0200A0
:1001500073905210B7B200009B82921073902230BD
:100160007350003097020000938242017390123462
:10017000732540F173002030B700008013010000A8
:1001800033D72000B703008093012000631A775E05
:10019000B70000801301100033D720009B0310002C
:1001A000939313029383F3FF9393E301930130003E
:1001B0006318775CB70000801301700033D720000C
:1001C0009B031000939313029383F3FF9393830194
:1001D000930140006316775AB70000801301E000D6
:1001E00033D720009B031000939313029383F3FFF4
:1001F000939313019301500063147758B700008064
:100200009B8010001301F00133D720009B031000E6
:10021000939313029383F3FF930160006312775665
:100220009300F0FF1301000033D720009303F0FF89
:1002300093017000631677549300F0FF13011000D0
:1002400033D720009B03F0FF9393F3039383F3FFD3
:1002500093018000631677529300F0FF1301700042
:1002600033D720009B031000939393039383F3FFF2
:1002700093019000631677509300F0FF1301E000A4
:1002800033D720009B031000939323039383F3FF42
:100290009301A0006316774E9300F0FF1301F00165
:1002A00033D720009B031000939313029383F3FF33
:1002B0009301B0006316774CB72021219B80101268
:1002C0001301000033D72000B72321219B83131291
:1002D0009301C0006316774AB72021219B8010123A
:1002E0001301100033D72000B79390109B830309AC
:1002F0009301D00063167748B72021219B8010120C
:100300001301700033D72000B74342009B8323249E
:100310009301E00063167746B72021219B801012DD
:100320001301E00033D72000B78300009B834348CC
:100330009301F00063167744B72021219B801012AF
:100340001301F00133D72000930300009301000153
:1003500063187742B72021219B801012130100FC03
:1003600033D72000B72321219B831312930110015F
:1003700063187740B72021219B801012130110FCD5
:1003800033D72000B79390109B830309930120017A
:100390006318773EB72021219B801012130170FC57
:1003A00033D72000B74342009B83232493013001BD
:1003B0006318773CB72021219B8010121301E0FCC9
:1003C00033D72000B78300009B834348930140014B
:1003D0006318773AB72021219B8010121301F0FF98
:1003E00033D720009303000093015001631A77383C
:1003F0009B0010009390F00113017000B3D0200017
:10040000B703000193016001639C70369B001000EC
:100410009390F0011301E00033D12000B7030200F4
:1004200093017001631E713493007000B3D010000B
:100430009303000093018001639470341302000061
:100440009B0010009390F0011301700033D720003F
:10045000130307001302120093022000E31252FE5E
:10046000B703000193019001631C73301302000075
:100470009B0010009390F0011301E00033D720009F
:100480001300000013030700130212009302200060
:10049000E31052FEB70302009301A0016312732E12
:1004A000130200009B0010009390F0011301F00173
:1004B00033D72000130000001300000013030700CF
:1004C0001302120093022000E31E52FC930310005B
:1004D0009301B0016316732A130200009B00100001
:1004E0009390F0011301700033D720001302120023
:1004F00093022000E31452FEB70300019301C001F0
:1005000063107728130200009B0010009390F00105
:100510001301E0001300000033D720001302120083
:1005200093022000E31252FEB70302009301D001B0
:1005300063187724130200009B0010009390F001D1
:100540001301F001130000001300000033D7200056
:100550001302120093022000E31052FE93031000D6
:100560009301E001631E7720130200009B0010003E
:100570009390F001130000001301700033D72000A6
:100580001302120093022000E31252FEB70300018F
:100590009301F0016316771E130200009B00100008
:1005A0009390F001130000001301E000130000001D
:1005B00033D720001302120093022000E31052FEF2
:1005C000B703020093010002631C771A13020000B4
:1005D0009B0010009390F001130000001300000036
:1005E0001301F00133D72000130212009302200000
:1005F000E31052FE93031000930110026312771868
:1006000013020000130170009B0010009390F00192
:1006100033D720001302120093022000E31452FE8D
:10062000B703000193012002631C7714130200003A
:100630001301E0009B0010009390F00113000000F4
:1006400033D720001302120093022000E31252FE5F
:10065000B703020093013002631477121302000003
:100660001301F0019B0010009390F00113000000B3
:100670001300000033D72000130212009302200061
:10068000E31052FE9303100093014002631A770EA9
:100690001302000013017000130000009B00100003
:1006A0009390F00133D72000130212009302200030
:1006B000E31252FEB7030001930150026312770C5C
:1006C000130200001301E000130000009B00100063
:1006D0009390F0011300000033D7200013021200A2
:1006E00093022000E31052FEB70302009301600260
:1006F00063187708130200001301F00113000000D3
:10070000130000009B0010009390F00133D72000ED
:100710001302120093022000E31052FE9303100014
:1007200093017002631E77049300F00033511000B0
:10073000930300009301800263147104930000028C
:1007400033D100009303000293019002631A7102F7
:10075000B3500000930300009301A0026392700263
:1007600093000040371100001B01018033D02000AE
:10077000930300009301B002631470006310300211
:100780000F00F00F638001009391110093E11100BD
:100790009308D00513850100730000000F00F00FCF
:1007A000930110009308D0051305000073000000AA
:0C07B000731000C00000000000000000FA
:1010000000000000000000000000000000000000E0
:1010100000000000000000000000000000000000D0
:1010200000000000000000000000000000000000C0
:1010300000000000000000000000000000000000B0
:081040000000000000000000A8
:040000058000000077
:00000001FF
